:100000000C943C020C9474020C9474020C947402D0
:100010000C9474020C9474020C9474020C94740288
:100020000C9474020C9474020C945A160C940F15D0
:100030000C94CD170C9474020C9474020C947402FA
:100040000C9474020C9474020C9474020C94740258
:100050000C9474020C948C170C9474020C9474021B
:100060000C9474020C9474020C9474020C94740238
:100070000C9474020C9474020C9474020C94740228
:100080000C9474020C9474020C9474020C94740218
:100090000C9474020C9474020C9474020C94740208
:1000A0000C9474020C9474020C947402081C2F1C9F
:1000B000C71D2F1CC71D771C9A1CC71D891D9C1DA1
:1000C00068026C02700268016C01700168046C04C3
:1000D00069026D02710269016D01710169046D04AB
:1000E0006A026E0272026A016E0172016A046E0493
:1000F0006B026F0273026B016F0173016B046F047B
:1001000000010101010101010101020202020202DA
:1001100002020203030303030303030404040404AD
:100120000404050505050506060606060707070774
:100130000708080808090909090A0A0A0B0B0B0C29
:100140000C0C0D0D0D0E0E0E0F0F0F1010111111C6
:100150001212131314141515161617171818191947
:100160001A1A1B1B1C1D1D1E1E1F202021222223AC
:100170002424252626272829292A2B2C2D2D2E2FED
:1001800030313232333435363738393A3B3C3D3E04
:100190003F404142434445464748494A4C4D4E4FF3
:1001A00050515354555658595A5B5D5E5F616264B5
:1001B000656668696B6C6D6F7072737577787A7B42
:1001C0007D7E8082838587888A8C8E8F9193959699
:1001D000989A9C9EA0A2A3A5A7A9ABADAFB1B3B5B9
:1001E000B7BABCBEC0C2C4C6C9CBCDCFD1D4D6D895
:1001F000DBDDDFE2E4E7E9EBEEF0F3F5F8FAFDFF33
:1002000000546474005565750056667600273747BC
:10021000005C6C7C005D6D7D005E6E7E002F3F4F4C
:10022000008494A4008595A5008696A6008797A7CC
:10023000008C9CAC008D9DAD008E9EAE008F9FAF5C
:100240000028384800293949002A3A4A002B3B4BFC
:10025000003040500031415100324252003343538C
:10026000008898A8008999A9005A6A7A005B6B7B7C
:100270000090A0B00091A1B100627282006373830C
:10028000000000000000000000000000000000006E
:10029000000000000000000000000000000000005E
:1002A000000000000000000000000000000000004E
:1002B000000000000000000000000000000000003E
:1002C000000000000000000000000000000000002E
:1002D000000000000000000000000000000000001E
:1002E000000000000000000000000000000000000E
:1002F00000000000000000000000000000000000FE
:1003000000000000000000000000000000000000ED
:1003100000000000000000000000000000000000DD
:1003200000000000000000000000000000000000CD
:1003300000000000000000000000000000000000BD
:1003400000000000000000000000000000000000AD
:10035000000000000000000000000000000000009D
:10036000000000000000000000000000000000008D
:10037000000000000000000000000000000000007D
:1003800005010906A1018506050719E029E7150001
:1003900025019508750181020507190029EF15004F
:1003A000250195F0750181020508190129059505BA
:1003B00075019102950175039101C005010906A11E
:1003C00001050719E029E715002501950875018148
:1003D000029501750881010507190029FF150026FE
:1003E000FF00950675088100050819012905950586
:1003F00075019102950175039101C009023B00024C
:100400000100A0FA09040000010301010009211103
:1004100001000122400007058103080001090401D1
:10042000000103000000092111010001223B000727
:10043000058203200001120100020000000845436C
:10044000C02E01000102000116034F00700065007C
:100450006E004400650063006B0033003200000052
:1004600012034F00700065006E00440065006300D9
:100470006B0000000403090411241FBECFEFDAE073
:10048000DEBFCDBF04B603FE18C080911D0590915C
:100490001E05A0911F05B09120058730904BA74005
:1004A000B04B59F410921D0510921E0510921F05B5
:1004B00010922005E0E0F8E3099512E0A0E0B1E039
:1004C000E2E3F1E402C005900D92A037B107D9F73D
:1004D00025E0A0E7B2E001C01D92AD31B207E1F71F
:1004E0000E945B110C9497200C94000080E008950A
:1004F000CF92DF92EF92FF926C01EE24FF24C114A1
:10050000D104E104F10421F0C701B60120E101C0EA
:1005100020E0C72ED82EE92EFF24C114D104E10417
:10052000F10419F0285FC701B6016B017C0154E0AA
:10053000F694E794D794C7945A95D1F7C114D1048F
:10054000E104F10419F02C5FC701B6016B017C01D5
:1005500042E0F694E794D794C7944A95D1F7C11432
:10056000D104E104F10419F02E5FC701B601DC01EA
:10057000CB01B695A79597958795892B8A2B8B2BC1
:1005800009F02F5F822FFF90EF90DF90CF900895BA
:10059000F894E82FE295EF70F0E031A1282F2F704A
:1005A00081E090E001C0880F2A95EAF7982F909596
:1005B000932391A392A1892B82A378940895CF933A
:1005C00084E090E00E94CB1FC82F82E290E00E945E
:1005D000CB1F2C2F30E0A901582BCA01CF910895D1
:1005E00069EE7EEF80E090E00E94072060E082E00C
:1005F00090E00E94E91F60E083E090E00E94E91F24
:1006000010920B0410920C0410920D0410920E0420
:1006100060E084E090E00E94E91F60E082E290E008
:100620000E94E91F60E085E090E00E94E91F60E021
:1006300086E090E00E94E91F6FEF87E090E00E9463
:10064000E91F40E050E0BA0188E090E00E94FB1F03
:1006500060E08DE090E00E94E91F40E050E0BA01C8
:1006600088E190E00E94FB1F60E087E190E00E943B
:10067000E91F40E050E0BA018CE190E00E94FB1FCE
:1006800060E070E080E290E00E94072040E050E0EF
:10069000BA0188E190E00E94FB1F40E050E0BA01FF
:1006A0008FE090E00E94FB1F40E050E0BA0183E140
:1006B00090E00C94FB1FCF93C091BD0480910A047D
:1006C000C82BC093720240E250E067E972E082E713
:1006D00092E00E948A20892B19F180E2E2E7F2E0A1
:1006E000A7E9B2E001900D928A95E1F7E091C1048B
:1006F000F091C2043097A1F080911201882349F053
:100700008091C80487FF05C0C093730286E0809380
:1007100072020280F381E02D82E792E0CF9109948A
:10072000CF9108951092BD0480911201882331F079
:100730008091C80487FF02C08EE101C086E0E4E733
:10074000F2E0DF011D928A95E9F710920A040C94F9
:100750005B03882341F080959091BD0489238093A9
:10076000BD040C945B030895882309F451C09CEFE9
:10077000980F913A30F4682F82E792E00E94F617C2
:1007800014C090E2980F983090F4877021E030E028
:10079000A90102C0440F551F8A95E2F7CA0180954E
:1007A0009091BD0489238093BD040C945B039BE569
:1007B000980F9330A0F48091930290919402892B2A
:1007C00039F11092940210929302E091C104F091D9
:1007D000C2043097E9F00680F781E02D16C0885AF0
:1007E0008731B0F48091950290919602892B81F027
:1007F0001092960210929502E091C104F091C20409
:10080000309731F00084F185E02D80E090E009948C
:100810000895CF93882309F453C09CEF980F913A21
:10082000C8F5C82F809112018823E1F08091C80497
:1008300087FF18C0EC2FE695E695E695F0E0EE58B8
:10084000FD4F8281282F30E04C2F477081E090E0EF
:1008500002C0880F991F4A95E2F782239323892BC0
:1008600061F412C0E4E7F2E08AE792E02191C21756
:1008700021F08E179F07D1F707C06C2F82E792E017
:100880000E94F6170E945B036C2F82E792E00E94A1
:100890001E1813C090E2980F983090F4877021E0F2
:1008A00030E0A90102C0440F551F8A95E2F7CA0142
:1008B0009091BD04892B8093BD04CF910C945B0370
:1008C000CF910895FF920F931F93CF93DF93CDB7EE
:1008D000DEB72F970FB6F894DEBF0FBECDBF4B87A4
:1008E0005C87F62E6D877E878F87611110920A04D0
:1008F00085E0FE013B96DE01169601900D928A95E9
:10090000E1F70E811F8189859A85892B31F01F3F80
:1009100031F481E00F3F19F403C081E001C080E0B1
:1009200080FD40C360910B0470910C0480910D0414
:1009300090910E040E947802E12FF0E024E0829F63
:10094000E00DF11D112423E0EE0FFF1F2A95E1F7C2
:10095000E00FF11DEE0FFF1FCF0180549F4FFC01F0
:1009600005911491043F4CE5140761F190F4093DA1
:100970004CE51407E9F00A3D2CE51207A9F1083D02
:100980004CE51407B9F506E221EE41EE68ED7CE591
:1009900014C0063F2CE5120709F1D0F0073F2CE503
:1009A000120741F507E225EE46EE67EF7CE505C04C
:1009B00007E225EE45EE69ED7CE5CE0106960E9444
:1009C0005F18F0C206E221EE40EE64EF7CE5F5CF61
:1009D00007E225EE44EE65EF7CE5EFCF06E221EE7F
:1009E00042EE66EF7CE5E9CF08E221E045EE6AEDF4
:1009F0007CE5E3CFF1101092C0042885222309F48E
:100A00005AC104304DE5140760F40B3F2CE5120782
:100A100088F4980122503C452431310508F035C155
:100A200009C002364DE5140729F0063A2DE51207F4
:100A300009F02BC10E94DF029093C9048093C8047F
:100A400001314CE5140709F4C6C008F042C0093072
:100A50009CE5190709F49BC000F505304CE5140727
:100A600009F485C078F403309CE5190709F478C0CF
:100A700008F07AC002301C4509F0F7C08091C80424
:100A80008160F1C007308CE5180709F478C008F0E0
:100A90007AC08091C8048061E6C00D302CE5120751
:100AA00009F487C058F40B308CE5180709F479C0B5
:100AB00008F07BC08091C80488606FC00F302CE5BF
:100AC000120709F480C008F082C08091C804877FB3
:100AD000CAC00E3F8CE5180709F471C000F5053156
:100AE0002CE5120709F485C068F403318CE518077A
:100AF00009F475C008F095C00E9492038091C80463
:100B00008F77B1C00C3F2CE51207A9F108F054C053
:100B10000B3F1C4509F0A9C08091C90440C00230B8
:100B20009DE5190709F489C058F401154DE514072E
:100B300009F45AC008F069C08091C90482602FC0CE
:100B400002369DE5190709F47EC0063A2DE5120725
:100B500009F483C003301D4509F087C060E06EC012
:100B60008091C80482607FC08091C80416C08091C3
:100B7000C804886078C08091C90482604FC08091A9
:100B8000C804806270C08091C80480646CC00E94F8
:100B900092038091C804806866C0846064C08160EC
:100BA0003DC08091C8048E7F5EC08091C8048D7F57
:100BB0005AC08091C80416C08091C90418C08091A1
:100BC000C9048D7F2BC08091C8048F7E4CC080915A
:100BD000C8048F7D48C08091C8048F7B44C0809139
:100BE000C804877F8B7F3FC08091C9048D7F8E7F33
:100BF00015C08091C80482FB222720F991E092273A
:100C000090FB82F990FB83F92EC08091C904982F44
:100C1000909591708E7F892B90FB81F98093C90408
:100C200024C00E9492038091C80487FB222720F9E8
:100C300091E0922790FB87F916C061E08EE090E08A
:100C40000E94E91F12C08091C80484FB222720F96A
:100C500091E0922790FB84F906C08091C804982FF8
:100C6000909590FB80F98093C8046091C80410911E
:100C7000C90484E090E00E94E91F612F82E290E0C5
:100C80000E94E91F0E9492038DC106312CE51207D4
:100C900021F58091BD048A7A91E009F490E0909367
:100CA0009202882311F065E301C069E282E792E0D5
:100CB0000E941E180FC006314CE5140709F046C00B
:100CC00080919202882309F463C165E382E792E090
:100CD0000E94F6170E945B0365C101154CE51407DD
:100CE00031F00F3D1C45B9F50E94F0025BC10E9436
:100CF00092034FE78AE196E0415080409040E1F74F
:100D000000C0000081E08093E00080E28093D80082
:100D10001092C9008FE097E20197F1F700C0000040
:100D200087E090EBDC0180931D0590931E05A09356
:100D30001F05B09320059CE088E10FB6F894A895B4
:100D4000809360000FBE90936000FFCF033C2CE5C2
:100D5000120708F01FC1FC0125913491C901223806
:100D6000310539F44091C80440FD0CC141FD0AC170
:100D700012C02338310508F0B0C02133310509F421
:100D800088C008F09BC02932310509F489C02A3295
:100D9000310509F48CC0283E310568F4203E310548
:100DA00080F42130310569F050F024503109213AA6
:100DB000310538F004C03A9521153F4110F080E02C
:100DC00090E0082F9032E0F5192F1F70892F807F57
:100DD00011F01295107F88858823C9F0112399F0AE
:100DE00080E2800F883010F0011106C08091BD04B0
:100DF000182B1093BD0405C080910A04182B109382
:100E00000A040E945B03802F0E94090419C0802FEE
:100E10000E94B4031123A1F0109580E2800F883066
:100E200010F0011106C08091BD0418231093BD0479
:100E300005C080910A04182310930A040E945B03E2
:100E400085E0FE013696DE01119601900D928A959D
:100E5000E1F760910B0470910C0480910D04909166
:100E60000E040E947802EA81F0E094E0899FE00D90
:100E7000F11D112483E0EE0FFF1F8A95E1F78981B0
:100E8000E80FF11DEE0FFF1FE054FF4F8591949185
:100E900089C02091C80426FF94CF8AE290E091CFC8
:100EA0002091C80425FF8DCF85E390E08ACF209163
:100EB000C80426FF86CF81E390E083CF2533310538
:100EC00039F42091C80425FF7CCF89E290E079CFE6
:100ED0002933310509F446CF5ECF233E310579F43D
:100EE0008091C80482FD4BC08091C90480FD4AC036
:100EF0008091C80484FD63CF83EE90E062CF243EEE
:100F00003105A8F4203E310549F42091C80420FDA4
:100F100033C02091C90420FF54CFEACF223E3105CF
:100F200009F039CF2091C80422FF4BCFE1CF263EF4
:100F3000310559F42091C80423FF43CF8091C804A0
:100F400084FD3DCF87EE90E03CCF273E310559F43C
:100F50008091C80483FD19C08091C90481FFEECF40
:100F600084EE90E02ECF243E310509F014CF20917D
:100F7000C90421FF26CFE2CF89E390E022CF82EEA1
:100F800090E01FCF80EE90E01CCF86EE90E019CF6E
:100F900069E29CCE073D4CE5140720F00E351D4557
:100FA00009F0D9CE2F960FB6F894DEBF0FBECDBF95
:100FB000DF91CF911F910F91FF9008959F92AF9273
:100FC000BF92CF92DF92EF92FF920F931F93CF9336
:100FD000DF9300D000D0CDB7DEB719821A821B8212
:100FE0001C820CE111E0AE014F5F5F4F7A015A01A4
:100FF000CC24C394D12CF80180818F3F09F441C0E7
:10100000F894E82FE295EF70F0E021A18F70A6012F
:1010100002C0440F551F8A95E2F7CA01922F982B00
:1010200091A392A18095892382A3789400C0E0E2E5
:10103000F1E0912C31E021912F3F89F0A22FA29570
:10104000AF70B0E090968C9190E02F7002C09595B3
:1010500087952A95E2F780FD02C0832F01C080E0CA
:10106000982A330F51E0E832F50729F7F80180811B
:101070008F3F11F00E94C802F0E5FA95F1F7F701F1
:1010800090820F5F1F4FFFEFEF1AFF0A41E000321F
:10109000140709F0B0CF44E050E0B50186E094E0D9
:1010A0000E948A2011E0009709F410E0892BA9F032
:1010B00089819A81AB81BC81809306049093070457
:1010C000A0930804B093090481E08093B9020E94C0
:1010D000C1179093B8028093B7028091B902882318
:1010E000D1F08091B7029091B8020E94B217059793
:1010F00090F08091060480930F0480910704809300
:101100001004809108048093110480910904809355
:1011100012041092B902812F0F900F900F900F9030
:10112000DF91CF911F910F91FF90EF90DF90CF90C3
:10113000BF90AF909F900895E42FF0E0EE0FFF1F57
:10114000E05BFE4F9081921B97FD9195292F38E12E
:10115000239F212D1124620F08950F931F9310E0F8
:10116000F801EE0FFF1FE05BFE4F9081905797FD57
:101170009195000F111FF801E05DFE4FE1A1F0E035
:10118000B097DF01AA0FBB1F8D010E0F1F1F200399
:10119000D001219FB00D1124E8E3F0E0E91BF10933
:1011A00097FDF3959F01220F331F89010E0F1F1F1B
:1011B00040039001419F300D11242A0F3B1F37FF40
:1011C00002C021583F4F220F232F221F330B620FE3
:1011D0001F910F9108950C94B6132091150530E1DD
:1011E000230F08F42FEF60E1822F90E00E94C110DE
:1011F000BC0188EB9BE00E94421F80E090E00895D4
:101200000F931F93CF93DF93D62F072F182FC42F41
:10121000822F0E943110EC2FF0E0EE0FFF1FE05BF9
:10122000FE4F90819058890F87FD8195880F682F18
:101230002CE0629F612D11246D0F702F812FDF91A3
:10124000CF911F910F9108950C946F135F926F923D
:101250007F928F929F92AF92BF92CF92DF92EF9246
:10126000FF920F931F93CF93DF93D82F8091170195
:101270008D130DC020911105237030E040911601AF
:1012800050E081E02417350719F480E001C081E0C7
:101290008170809315018091160590911401981723
:1012A00039F08093140140E060E080E00E94EB0898
:1012B000DF30F9F48FED9EE00E946319C82F05C05E
:1012C000C1E0EFE5EF1508F48AC0809113018F5F4C
:1012D00080931301C111D9C482E0809318018091D9
:1012E00015018111D2C4D111D0C483E080931801BB
:1012F000CCC4D03108F074C1D73019F48EE09FE02F
:10130000DBCFD83008F047C1D33009F03BC0C091E3
:10131000130184E1C89FC02D112414E11C0F113664
:1013200008F010E6D0901305C09014052091150523
:1013300000E4029F012D1124C11708F040C0EC2EDB
:10134000F12CF701E05FFD4F90818091140189231A
:10135000B9F0F701EE0FFF1FE05DFE4F81A182950E
:101360008F7060911205809F600D11247D2D8C2D52
:101370000E94CB10462F282F672FC7010E942409F7
:10138000CF5FDACFD43008F07AC0D130E9F4809161
:101390001301C4E18C9FC02D112414E11C0F1136E0
:1013A00008F010E660911205709113058091140504
:1013B0000E94CB10062FF72EE82EC11790F0C1E047
:1013C000103608F482CF0BC0D230E8F480911501BA
:1013D000882329F040E060E080E00E94EB08C0E054
:1013E00074CFEC2FF0E0DF01A05FBD4F8C919091A6
:1013F0001401982331F02E2D402F6F2DCF010E9424
:101400002409CF5FDACFC091130184E1C89FC02DBA
:10141000112414E11C0F113608F010E6F0901305AA
:1014200000911405E0901205B701802F0E94CB10A7
:10143000D62EC72EB82E609115056E0D7F2D802FEC
:101440000E94CB10062FF72EE82EC11708F0B7CF59
:101450008C2F90E0FC01E05FFD4F30812091140162
:10146000232359F030FF04C02E2D402F6F2D03C0D1
:101470002B2D4D2D6C2D0E942409CF5FE6CFD5304A
:1014800009F044C0C091130184E1C89FC02D11240C
:1014900014E11C0F113608F010E6F09012050091CF
:1014A0001305E0901405609115056695669566959F
:1014B00080910D0590910E050E94C1100E9431107F
:1014C000805887FD8195880F282F3E2D239F212D41
:1014D0001124822F6F2D702F0E94CB10062FF72E14
:1014E000E82EC11708F06BCFEC2FF0E0DF01A05F12
:1014F000BD4F8C9190911401982331F02E2D402FE7
:101500006F2DCF010E942409CF5FEBCFD63008F0BA
:101510003FC0C091130184E1C89FC02D112414E184
:101520001C0F113608F010E6D0901305C09014057A
:101530002091150500E4029F012D1124C11708F028
:101540003ECFEC2EF12CF701E05FFD4F90818091B2
:1015500014018923D9F0F701EE0FFF1FE05BFE4F66
:101560006081069FB0011124B5E075956795BA9525
:10157000E1F780911205680F7D2D8C2D0E94CB1014
:10158000462F282F672FC7010E942409CF5FD6CF8F
:101590008AE39FE091CEDB3041F48DEB9FE002C007
:1015A00089ED9FE00E94121A89CEDC3060F4D930B8
:1015B00019F484EF9FE004C0DA3090F783E190E102
:1015C0000E948E1A7BCEDD3019F483E09FE074CE4A
:1015D000DE3018F48CE09FE06FCE8AEF9EE06CCE98
:1015E000D73109F03FC08091150181111EC0609173
:1015F000150520E1620F08F46FEF80910D059091C1
:101600000E050E94C1106AE070E00E94421F892B03
:1016100009F0E5CE0E94A21F60E670E00E947020F3
:10162000609114010E941D19DACE8091130104E12A
:10163000809F002D112474E1F72EF00E80E68F15A7
:1016400010F460E6F62E10E0CF2CD12C0C151D0501
:101650000CF036CE60911401C8010E941D190F5F75
:101660001F4FF4CFD83118F5D33119F488E99FE032
:1016700099CFD43168F4D13119F488E990E1A0CF41
:10168000D23118F480ED9EE08DCF8CEA9FE098CFA8
:10169000D53119F480E79EE004C0D63128F482EAFF
:1016A0009EE00E94B1190ACE8DEA98E0FACFDB31B4
:1016B00019F48CE998E000CEDC3108F091C0D93102
:1016C00009F044C0C091130184E1C89FC02D1124CA
:1016D00014E11C0F113608F010E6F090130500918C
:1016E0001405E0901205609115056695669566955E
:1016F00080910D0590910E050E94C1100E9431103D
:10170000805887FD8195880F682F2CE0629F612D9E
:1017100011246E0D7F2D802F0E94CB10062FF72EE7
:10172000E82EC11708F04BCEEC2FF0E0DF01A05FF0
:10173000BD4F8C9190911401982331F02E2D402FA4
:101740006F2DCF010E942409CF5FEBCFDA3108F073
:1017500044C08091150181111EC06091150520E1E2
:10176000620F08F46FEF80910D0590910E050E94B5
:10177000C11065E070E00E94421F892B09F02FCE56
:101780000E94A21F60E670E00E9470206091140128
:101790000E94F61824CE8091130104E1809F002D51
:1017A000112454E1F52EF00EF0E6FF1510F440E69A
:1017B000F42E10E0CF2CD12C0C151D0544F46091B3
:1017C0001401C8010E94F6180F5F1F4FF5CFC1E04A
:1017D0002FE52F1508F079CD02CE80E099E06CCD91
:1017E000DD3109F0E5C04091DE035091DF036091E7
:1017F000E0037091E10380910D0590910E05A09199
:101800000F05B091100584179507A607B70708F4D0
:10181000E6CD8091150181110DC080911301C4E1C5
:101820008C9FC02D112404E10C0F013608F454C024
:1018300000E652C040E060E080E00E94EB083EEB32
:10184000E32E32E0F32E00E010E0CFE70E945210CA
:1018500081FF05C0F7011082118212821DC00E9413
:101860005210B82E0E9452108695782F2C2F720F8E
:1018700008F47FEFC801880F991F800F911FFC01AA
:10188000E254FD4F6F016B2D809114050E94CB1027
:10189000F6016083718382830F5F1F4FF3E0EF0EC9
:1018A000F11C0036110591F6B8CF8C2F90E0FC01A9
:1018B000E05FFD4F308120911401232361F0FC0192
:1018C000EE0FFF1FE80FF91FE254FD4F2281408108
:1018D00061810E942409CF5FC01738F3C1E0003650
:1018E00008F0C0E0003608F4F0CC20E010E0015031
:1018F0001109822F90E080179107CCF4AC01440FBE
:10190000551F480F591F42545D4F0196FC01EE0FC1
:10191000FF1F8E0F9F1FFC01E254FD4F80819181BC
:10192000A281FA0180839183A2832F5FE2CF0E947C
:1019300052107801EE0CFF1C81FF09C00E0D1F1D17
:10194000F801E254FD4F10821182128218C00E94E9
:101950005210D82E0E9452108695782F2FE7720FC2
:1019600008F47FEF0E0D1F1D02541D4F6D2D809149
:1019700014050E94CB10F8016083718382830E945A
:10198000ED0800910D0510910E0520910F05309185
:101990001005DC01CB01800F911FA21FB31F8093A4
:1019A000DE039093DF03A093E003B093E1038DCCBB
:1019B000DD3108F06DC04091BA025091BB026091D8
:1019C000BC027091BD0280910D0590910E05A09111
:1019D0000F05B091100584179507A607B70708F4FF
:1019E000FECC0E945210C82F0E94521090E6891B14
:1019F000F0F7890F082F10E0F801E05FFD4F90919C
:101A000014018081892309F441C0C1FF04C020E092
:101A100040E060E013C00E945210C82F0E94521094
:101A20008695782F2FE7720F08F47FEF6C2F809147
:101A300014050E94CB10462F282F672FC8010E9443
:101A400024092091150530E1230F08F42FEF60E100
:101A5000822F90E00E94C110BC0184EF91E00E94AF
:101A6000421F80910D0590910E05A0910F05B09138
:101A70001005860F971FA11DB11D8093BA02909388
:101A8000BB02A093BC02B093BD02A9CCC1E01DCCA7
:101A9000DE3109F0C1C0409102045091030460910D
:101AA00004047091050480910D0590910E05A0919C
:101AB0000F05B091100584179507A607B70708F41E
:101AC0008ECC80911501882329F040E060E080E011
:101AD0000E94EB0860911205709113058091140526
:101AE0000E94CB10C62F772E682E02EE13E050E333
:101AF000E52E51E0F52E62E0A62E64E0B62E4701F9
:101B0000680133E0532EF6018081F401882329F027
:101B10008081262D4C2F672D04C0808120E040E07D
:101B200060E090E00E942409F601818181936F01B9
:101B30005A94FFEF8F1A9F0A5110E5CF47016801B1
:101B400043E0542EF6018781F401882329F0878130
:101B5000262D4C2F672D04C0878120E040E060E0F7
:101B600090E00E942409F601868187835A94F1E06F
:101B7000CF1AD10821E0821A91085110E3CFF80161
:101B80008481F701882329F08481262D4C2F672D2D
:101B900004C0848120E040E060E090E00E942409DD
:101BA000F8018381F701882329F08381262D4C2FAA
:101BB000672D04C0838120E040E060E090E00E9457
:101BC00024090E945210837091E009F090E0F8011E
:101BD00093839483085F1F4FF8E0EF0EF11CA0166B
:101BE000B10609F08CCF0E94ED0800910D0510910F
:101BF0000E0520910F0530911005DC01CB01800FFF
:101C0000911FA21FB31F8093020490930304A0931B
:101C10000404B0930504E3CBDF3F89F580910D0503
:101C200090910E05A0910F05B091100588279C702A
:101C3000AA27BB272AE0B695A795979587952A9559
:101C4000D1F782309105A105B10571F0833091057E
:101C5000A105B10569F040E00197A105B10511F0BA
:101C600060E008C064E102C044E160E080E003C0DD
:101C700044E164E184E10E94EB0882E037CB80918B
:101C800013018F5F8093130127CBDF91CF911F91B9
:101C90000F91FF90EF90DF90CF90BF90AF909F900B
:101CA0008F907F906F905F900895E1E1F5E08DE473
:101CB00080838091190190911A01A0911B01818369
:101CC0009283A3838FE784838FEF858346E050E080
:101CD0006CE170E0CF010E94D91F10921B0508959E
:101CE0000F931F93522F10E0F801EE0FFF1FE05DDE
:101CF000FE4FE1A1F0E0B097EE0FFF1F9F015203EE
:101D0000D001539FB00D1124000F111FF801E05BAB
:101D1000FE4F008110E000571109000F111F400312
:101D20009001419F300D11242A0F3B1F37FF02C045
:101D300021583F4F220F232F221F330B620F1F9179
:101D40000F9108950F931F93522F10E0F801EE0F9B
:101D5000FF1FE05DFE4FE1A1F0E0B0979F0152034D
:101D6000D001539FB00D1124000F111FF801E05B4B
:101D7000FE4F008110E00057110940039001419F80
:101D8000300D11242A0F3B1F37FF02C021583F4F4F
:101D9000220F232F221F330B620F1F910F910895E3
:101DA000EF920F931F9393E0099F800111241595E3
:101DB00007956E2D600F1F910F91EF900895A22F40
:101DC00050E0FA01EE0FFF1FE05DFE4F91A190522F
:101DD00097FD9195440F551FFA01E05BFE4F30814E
:101DE000232F30E02A1B3109290F311D97FD3A9529
:101DF000620F0895E42FF0E0EE0FFF1FE05DFE4F4D
:101E000061A1621B0895E42FF0E0EE0FFF1FE05B7D
:101E1000FE4F6081621B0895622F0895E42FF0E069
:101E2000EE0FFF1FE05BFE4F408134EE439F412DDC
:101E30001124E82FF0E050E0445E5F4FDA01A21B6E
:101E4000B1099D01B7FF03C031952195310993E098
:101E5000220F331F9A95E1F7AF01421B530B9A01F2
:101E600057FF02C020E030E0582F259F212D11247C
:101E7000822F0895E42FF0E0EE0FFF1FE05BFE4F8E
:101E8000408134EE439F412D1124E72FF0E050E0D4
:101E9000445E5F4FDA01A21BB1099D01B7FF03C089
:101EA00031952195310993E0220F331F9A95E1F77F
:101EB000AF01421B530B9A0157FF02C020E030E0F4
:101EC000279F212D1124722F0895FC019B0100975B
:101ED00021F477FF2BC080E80895AC0197FF04C080
:101EE00044275527481B590BB901640F751F37FD4F
:101EF0000CC0241B350BC901A5E0880F991FAA95BA
:101F0000E1F70E94702080E20CC0CB0165E0880FF1
:101F1000991F6A95E1F7BA01621B730B0E9470204A
:101F200080E6861BF7FF03C08195089580E0089541
:101F3000EF920F93CF93DF93D72FC82FC9010E19BC
:101F4000BA010E94650F602F681B7D2F8C2FDF91D7
:101F5000CF910F91EF9008950F93CF93DF93D72FE9
:101F6000C82FC901BA010E94650F682F600F7D2F2D
:101F70008C2FDF91CF910F910895EF920F931F93C4
:101F8000CF93DF93D62FC72F182FC9010E19010F3A
:101F9000BA010E94650F081B202F219F212D1124BB
:101FA000822F6D2F7C2FDF91CF911F910F91EF909A
:101FB0000895EF920F931F93CF93DF93D62F172F90
:101FC000C82FC9010E19070FBA010E94650F702FA3
:101FD000781B719F712D11246D2F8C2FDF91CF9164
:101FE0001F910F91EF900895FF920F931F93CF933E
:101FF000DF93F62ED72F182FC901C12FC01BBA01AE
:102000000E94650F982F990F890FC81B2C2F219FB5
:10201000212D1124822F6F2D7D2FDF91CF911F91C4
:102020000F91FF900895FF920F931F93CF93DF932B
:10203000F62E172FD82FC901C72FC01BBA010E9437
:10204000650F982F990F890F7C2F781B719F712D29
:1020500011246F2D8D2FDF91CF911F910F91FF9044
:102060000895482F982F46FD9095E92FEF739F70A4
:1020700046FD9F5FE295EF70EE0FF0E0E85DFE4FEA
:102080002181299F802D212D112482958F702295E9
:10209000207F822B3081982F930F892F47FD8195C8
:1020A00080580895409110015091110125E038E0C9
:1020B000429FC001439F900D529F900D1124875E57
:1020C000994C9093110180931001890F0895BC01E0
:1020D0008230910508F40895613E8EE1780748F456
:1020E0009B0195E0369527959A95E1F748E0420FD8
:1020F00001C04FEF91E0242F30E0290F311D3595BD
:102100002795229FF001239FF00DF00D11246E17EB
:102110007F0718F44FEF420F04C02F3F39F091E0D2
:10212000920F491740F78FEF890F08958FEF0895A9
:102130000F93CF93DF93D72FC82F47FD4195E8E347
:10214000F0E0CF01841B910947FD9395889FB00172
:10215000899F700D700D1124229FC001239F900D47
:10216000900D1124860F971F0E946710682F660F2D
:10217000860F682F600F7D2F8C2FDF91CF910F91ED
:10218000089520E030E0869F212D969F200D311D7F
:102190001124C9010895CF92DF92EF92FF920F931D
:1021A0001F93CF93DF93F62E472FE82FF0E07111A6
:1021B00006C0E050FF4F8491782F682F73C0272FFF
:1021C00030E0E050FF4FE491FE2F0E2F10E056E07C
:1021D000659FC0011124CFEFD0E0BE010E94421FD5
:1021E0005BEA5603C001579F900D11248F0D911D7E
:1021F0008F0D911D982F990F980F7E01E21AF30A07
:10220000E09ED001E19EB00DF09EB00D11248B2F09
:10221000499FA0011124452F55277E01E41AF50A94
:10222000E09EA001E19E500DF09E500D11246E0124
:10223000C91AD108C29E7001C39EF00CD29EF00C48
:1022400011242F2D3327C21BD30BC09F9001C19F98
:10225000300DD09F300D1124932F6230710591F015
:1022600048F461157105E1F061307105B9F49E2FF4
:10227000E52F16C06430710569F040F066307105D5
:1022800079F00CC09E2FEB2F832F0AC0EB2F8F2FDE
:10229000952F06C09B2F8E2FE32F02C09B2F852FDB
:1022A0007E2F692FDF91CF911F910F91FF90EF90BB
:1022B000DF90CF900895CF93DF93CDB7DEB72A9705
:1022C0000FB6F894DEBF0FBECDBF84B7877F84BF43
:1022D0000FB6F894A89580916000886180936000A3
:1022E000109260000FBE90E080E80FB6F8948093E3
:1022F0006100909361000FBE85B7806885BF85B788
:10230000806885BF86E792E09093710280937002A7
:10231000819A8998529A5A9A53985B980E945315B9
:102320000E94F9158091E20084608093E200789425
:102330008091EF048823A1F01091E9001F70909123
:10234000EC00892F817090FD80E8182B1092E90035
:102350008091E80083FD0E94221B1F701093E9000A
:1023600082E084BD93E095BD9DE797BD80936E00AC
:102370000CE111E030E2E32E31E0F32ED8018D9133
:102380008D018F3F11F00E94C802E016F106B1F7EF
:1023900000E211E0F80181918F018F3F11F00E945E
:1023A000C802F1E008321F07A9F784E0EFE0F4E08B
:1023B000DF01282F1D922A95E9F7E6E0F4E0DF011E
:1023C0001D928A95E9F780E090E00E94D31F893E34
:1023D0009E4F11F00E94F00282E090E00E94CB1F1D
:1023E000809313040E94DF029093C9048093C80471
:1023F00083E090E00E94CB1F90E0A0E0B0E08093EB
:102400000B0490930C04A0930D04B0930E0410924F
:102410000A040E945B030E94FA1380E090E00E948D
:10242000D31F893E9E4F21F00E94F0020E94550E5C
:1024300046E050E06CE170E081E195E00E94BB1F56
:1024400010921B05809111058C7F11F40E94550E8E
:102450006091C80460686093C8041091C90484E066
:1024600090E00E94E91F612F82E290E00E94E91F44
:1024700080911105837011F410921801809111055B
:102480008C7F81608093110584E091E09093C20479
:102490008093C10498E1C92ED12C20E4A22EEE2411
:1024A000E39482E0B82E8091EF04853009F05AC0A1
:1024B0008091EF04853009F04FC08091EF048430A3
:1024C00009F439C080911C05811105C00E942609BC
:1024D00080E00E94EF1DE0921C050E94FC1D80918F
:1024E0001C05811105C00E94260980E00E94EF1D95
:1024F000E0921C051092C3040FB6F894A895C09200
:1025000060000FBEA092600083B7817F846083BFAC
:1025100083B7816083BF7894889583B78E7F83BFAC
:102520000FB6F894A8958091600088618093600050
:10253000109260000FBE8091EE04882309F4B8CF9A
:102540000E94DE07EFE0F4E0819181116AC024E08F
:10255000E331F207C9F7ACCF0E9492030E945318EF
:1025600010921C050E94DE07882359F08FB7F8945B
:102570004091C4045091C5046091C6047091C70491
:102580008FBFAFE0B4E0E4E1F4E000E010E0302F12
:102590002D919191922721F180E0FF24F3944F2D0A
:1025A0004923D1F089833A832F2181E009F480E027
:1025B0008B830E94C1178160782F9D838C83498112
:1025C0005A816B818D810E946204F801EC5EFB4FA1
:1025D0008081F826F08219C08F5FFF0C8830F9F6F1
:1025E0000F5F1F4F0430110591F68FEF8E838F839D
:1025F00018860E94C1178160782F9A8789874E813B
:102600005F8168858A850E9462040E94FC1D0E9489
:10261000531890911804891709F445CF8093180432
:1026200040CF19BCB9BC09B400FEFDCF8091D800E1
:102630008F7D8093D8008091E00082608093E000DD
:102640008091E00081FDFCCF0E94920331CF08957C
:102650000895089508958091CC040895CF93DF9351
:1026600020911201222339F02091C80427FF03C0D2
:1026700060E222E002C068E021E02093E9002FEF51
:102680003091E800215035FD06C03AE63A95F1F761
:1026900000C02111F5CF2091E80025FF1DC0EC01FD
:1026A00080911201811105C040E050E068E070E0C7
:1026B00003C070E040E050E0CE010E94F61A809125
:1026C000E8008E778093E80080E2FE01ADECB4E094
:1026D00001900D928A95E1F7DF91CF910895FF92D5
:1026E0000F931F93CF93DF9300D000D0CDB7DEB709
:1026F0008036910588F5122F042FF62EBC01660F47
:10270000771F660F771F60507E4F44E050E0CE0188
:1027100001960E94B21F898183704A81282F30E080
:1027200050E9859FC0011124835D9B4FFC01E40F9C
:10273000F11DB497F0824B81FC01E40FF11DB497B9
:1027400000834C81840F911DFC01B4971083F90123
:10275000E45DFB4F81E080830F900F900F900F900E
:10276000DF91CF911F910F91FF900895FF920F93EA
:102770001F93CF93DF93182F062FF42EC0E0D0E0E5
:102780002F2D402F612FCE010E946F132196C0364E
:10279000D105B1F7DF91CF911F910F91FF9008956F
:1027A0000F931F93CF9380912C04811106C0109238
:1027B0002C04CF911F910F9108950DE214E0C4E213
:1027C000C093F904EAEFF4E0D8018D91819385E09C
:1027D000EA30F807D1F724E630E041E150E069EF54
:1027E00074E088EE0E941B1FC05F005F1F4FC43B58
:1027F00039F7DDCF4F925F926F927F928F929F92C7
:10280000AF92BF92CF92DF92EF92FF920F931F93FE
:10281000CF93DF9300D000D0CDB7DEB70E94641E07
:102820006BE08DEF0E94EA1A60E08AE00E94EA1AEB
:102830008FE19EE40197F1F700C0000060E080E0C6
:102840000E94EA1A60E081E00E94EA1A60E086E0F5
:102850000E94EA1A60E08DEF0E94EA1A10E060E040
:10286000812F0E94EA1A1F5F1231C9F760E0812FA1
:102870000E94EA1A1F5F1432C9F760E0812F0E949C
:10288000EA1A1F5F143BC9F76BE08DEF0E94EA1A4A
:1028900061E08AE00E94EA1A60E08DEF0E94EA1A85
:1028A00000E012E070E8472E73E0572EE2E17E2E42
:1028B000F8E0CF2ED12CEE24E394F12C662463941F
:1028C00044E050E0B801CE0101960E94B21F4A8157
:1028D00050E0CA018497AB80B12CA4E2AA1AB108D7
:1028E000EC81F0E0B4979C0197FF02C0295F3F4F55
:1028F000A90163E0559547956A95E1F72981237011
:1029000030E0729EB001739E700D1124675E7B4FA4
:102910004B01840E911CB6010E947020A70102C0D9
:10292000440F551F8A95E2F7CA01D4019C91892B67
:102930008C93C501B7FC079653E0959587955A95FA
:10294000E1F7729EA001739E500D1124475E5B4F0C
:102950004A01880E911CC501B6010E947020A70192
:1029600002C0440F551F8A95E2F7CA01D4019C9119
:10297000892B8C93CF01F7FD079643E095958795BA
:102980004A95E1F7729EA001739E500D1124475E97
:102990005B4F5A01A80EB11CCF01B6010E947020F6
:1029A000F70102C0EE0FFF1F8A95E2F7CF01D501B4
:1029B0009C91892B8C93F901E55DFB4F60820C5F44
:1029C0001F4F4016510609F07BCF80912B048111D7
:1029D00017C010922B040F900F900F900F90DF9163
:1029E000CF911F910F91FF90EF90DF90CF90BF900C
:1029F000AF909F908F907F906F905F904F900895D1
:102A000089E1E82E84E0F82E10E0F70161917F0162
:102A1000812F0E94EA1A1F5F1231B9F7DACF1F9295
:102A20000F920FB60F9211242F933F934F935F9302
:102A30006F937F938F939F93AF93BF93CF93DF93C6
:102A4000EF93FF93C091E900CF708091EC00D82FF5
:102A5000D17080FDD0E81092E9008091F000877F6E
:102A60008093F00078940E94221B1092E9008091DC
:102A7000F00088608093F000CD2BCF70C093E90008
:102A8000FF91EF91DF91CF91BF91AF919F918F9186
:102A90007F916F915F914F913F912F910F900FBE5A
:102AA0000F901F901895E8EDF0E080818E7F808375
:102AB0001092E2001092DA001092E100A0EEB0E075
:102AC0008C9181608C9380818F77808319BCA7ED76
:102AD000B0E08C918E7F8C9380818F7E808310926A
:102AE000CA0408952091E4003091E50095E64091F4
:102AF000EC00842F817040FF23C08091E80080FDAE
:102B00001DC08091EF04882399F0853099F0809161
:102B1000EB0085FD11C04091E4005091E5002417C1
:102B2000350729F3915011F09A01E1CF84E008951F
:102B300082E0089583E0089581E0089580E008959B
:102B40004091E80042FFDDCF08958091F10487FFB6
:102B500011C08091E80082FD05C08091EF048111D1
:102B6000F8CF11C08091E8008B770BC08091EF0403
:102B7000882349F08091E80080FFF8CF8091E80039
:102B80008E778093E8000895982F973068F590939A
:102B9000E900981739F07091EC002091ED00509108
:102BA000F00003C0242F762F50E021FD02C09F5F6C
:102BB000ECCF3091EB003E7F3093EB003091ED0095
:102BC0003D7F3093ED003091EB0031603093EB00AE
:102BD0007093EC002093ED005093F0002091EE00F4
:102BE00027FDE5CF80E008958F708093E90081E0B4
:102BF0000895CF92DF92EF92FF920F931F93CF939E
:102C0000DF93C8EDD0E088818F7E8883E7EDF0E028
:102C100080818160808384E082BF81E08093CA04E8
:102C200088818E7F888302EE10E0F8011082109276
:102C3000DA0081EEC82ED12CF601108288818F77C0
:102C4000888388818068888388818F7D888319BC88
:102C50001092EF041092F0041092EE041092ED0422
:102C600090EEE92EF12CF70180818B7F80838881A3
:102C70008160888342E060E080E00E94C415F60134
:102C800080818E7F8083F801808181608083808154
:102C900088608083F70180818E7F80838881806156
:102CA0008883DF91CF911F910F91FF90EF90DF907C
:102CB000CF9008951F920F920FB60F9211242F9369
:102CC0003F934F935F936F937F938F939F93AF93B4
:102CD000BF93EF93FF938091E10082FF09C0809141
:102CE000E20082FF05C08091E1008B7F8093E100CC
:102CF0008091DA0080FF28C08091D80080FF24C036
:102D00008091DA008E7F8093DA008091D90019BC1F
:102D100080FF16C082E089BD09B400FEFDCF81E0CE
:102D20008093EF048091CA0481110EC00E94531554
:102D30000E94F9158091E20084608093E20004C053
:102D40001092EF041092CA048091E10080FF17C036
:102D50008091E20080FF13C08091E2008E7F80931B
:102D6000E2008091E20080618093E2008091D800CF
:102D700080628093D80019BC85E08093EF04809135
:102D8000E10084FF2FC08091E20084FF2BC019BCBA
:102D900082E089BD09B400FEFDCF8091D8008F7D0F
:102DA0008093D8008091E1008F7E8093E100809134
:102DB000E2008F7E8093E2008091E2008160809348
:102DC000E2008091F004882311F084E007C0809134
:102DD000E30087FD02C081E001C083E08093EF043F
:102DE0008091EF048091E10083FF27C08091E20091
:102DF00083FF23C08091E100877F8093E10082E020
:102E00008093EF041092F0048091E1008E7F809314
:102E1000E1008091E2008E7F8093E2008091E200E9
:102E200080618093E20042E060E080E00E94C4158F
:102E30008091F00088608093F000FF91EF91BF9146
:102E4000AF919F918F917F916F915F914F913F9142
:102E50002F910F900FBE0F901F9018952091F7049F
:102E60003091F8042617370748F06115710539F4D9
:102E70002091E8002E772093E80001C0B901FC0101
:102E800020E06115710579F18091EF048823F1F15B
:102E90008530F1F18091E80083FD3CC08091E8002D
:102EA00082FD2EC08091E80080FFEBCF2091F300DF
:102EB0008091F20090E0922B6115710551F08830FD
:102EC000910538F421912093F10061507109019628
:102ED000F3CF21E0089709F020E08091E8008E7799
:102EE0008093E800CECF2111CFCF0AC08091EF04AC
:102EF000882361F0853061F08091E80083FD0AC08D
:102F00008091E80082FFF2CF80E0089582E008958A
:102F100083E0089581E0089578941F920F920FB690
:102F20000F9211248F939F93AF93BF938091C4040A
:102F30009091C504A091C604B091C7040196A11D4B
:102F4000B11D8093C4049093C504A093C604B093AC
:102F5000C704BF91AF919F918F910F900FBE0F90BB
:102F60001F9018959C014FB7F8948091C4049091DC
:102F7000C504A091C604B091C7044FBF821B930B38
:102F800008952FB7F8948091C4049091C504A0913E
:102F9000C604B091C7042FBF08951F920F920FB6B9
:102FA0000F9211248F939F93AF93BF938091C3048B
:102FB000811113C08091C4049091C504A091C604EE
:102FC000B091C7044196A11DB11D8093C404909394
:102FD000C504A093C604B093C704BF91AF919F915D
:102FE0008F910F900FBE0F901F9018952091120196
:102FF0002223C9F02091C80427FF15C0262F26954B
:10300000269526952E31C8F4FC01E20FF11D67705C
:1030100081E090E001C0880F6A95EAF7809592817F
:10302000892382830895FC0106962281621301C0E0
:1030300012823196E817F907C1F70895209112011D
:103040002223C1F02091C80427FF14C0262F269503
:10305000269526952E3130F5FC01E20FF11D6770A3
:1030600081E090E001C0880F6A95EAF79281892B90
:1030700082830895FC0132962FEF30E0419164176E
:1030800089F02F3F19F4411101C0232F3F5F3630E3
:10309000A9F72F3F39F0FC01E20FF11D27FDFA954A
:1030A000628308950895E091C104F091C2043097BD
:1030B00021F00190F081E02D099480E00895EF92D5
:1030C000FF920F93CF93DF93C42FD22FFC01828105
:1030D000882301F14093C0040E94C1179093BF045C
:1030E0008093BE0480E28C0F883008F079C0C770EE
:1030F00081E090E001C0880FCA95EAF79091BD0485
:10310000892B8093BD04DF91CF910F91FF90EF90B9
:103110000C945B038091C004481351C08091BE049D
:103120009091BF040E94B217883C910508F047C0F7
:10313000CD17F9F080E28C0F883040F4C77081E041
:1031400001C0880FCA95EAF70E94A90380E28D0F9B
:10315000883078F42D2F277081E090E001C0880F2F
:103160002A95EAF79091BD04892B8093BD040E94B3
:103170005B03093319F0E12CF12C03C080E5E82E44
:10318000F12C802F0E940904E114F10451F08FEC1E
:1031900097E00197F1F700C0000091E0E91AF1080B
:1031A000F3CF802F0E94B40380E28D0F8830C0F4EB
:1031B000D77081E001C0880FDA95EAF70AC080E293
:1031C0008C0F883068F4C77081E001C0880FCA9501
:1031D000EAF7DF91CF910F91FF90EF900C94A90344
:1031E000DF91CF910F91FF90EF9008951F93CF93B0
:1031F000DF93FC01E05FFD4F20816223D1F0EC0101
:103200000E94A21F182F0E94A21F8F77782F20E8FC
:10321000720F08F47FEF612F809114050E94CB108C
:10322000462F282F672FCE01DF91CF911F910C944D
:103230002409DF91CF911F910895DF92EF92FF92C1
:103240000F931F93CF93DF93EC01FC01E05FFD4FE1
:103250009081692381F1D09013050091140510919C
:103260001205E12EF12C0E94A21F282FC7018C54B9
:103270009F4F68E671E00E9470208E199F0997FDAC
:10328000039695958795959587952370612F289F2F
:10329000600D11247D2D802F0E94CB10462F282FEA
:1032A000672FCE01DF91CF911F910F91FF90EF908B
:1032B000DF900C942409DF91CF911F910F91FF9023
:1032C000EF90DF900895DF92EF92FF920F931F939C
:1032D000CF93DF938C01C091130184E1C89FC02D6F
:1032E0001124D4E1DC0FD13608F0D0E66091150549
:1032F0006695669521E0620F08F46FEF80910D05E9
:1033000090910E050E94C110D82ECD17F0F4EC2E2E
:10331000F12CF701E05FFD4F90818091140189232A
:1033200091F06091120570911305809114052D2D77
:103330004C2FF80109950E94CB10462F282F672F9C
:10334000C7010E942409CF5FE0CF81E0D03608F0AA
:1033500080E0DF91CF911F910F91FF90EF90DF9070
:1033600008959F92AF92BF92CF92DF92EF92FF9219
:103370000F931F93CF93DF936C01C091130184E1EE
:10338000C89FC02D1124D4E1DC0FD13608F0D0E65F
:10339000609115056695669580910D0590910E05D5
:1033A0000E94C110182F80E4810F0E94311090E814
:1033B000F92EF80E812F0E94311020E8922E980EDF
:1033C000CD1700F5AC2EB12CF501E05FFD4F9081DB
:1033D000809114018923A1F0609112057091130569
:1033E00080911405E12E0C2F292D4F2DF601099502
:1033F0000E94CB10462F282F672FC5010E94240959
:10340000CF5FDECF81E0D03608F080E0DF91CF9152
:103410001F910F91FF90EF90DF90CF90BF90AF90F2
:103420009F9008956F927F928F929F92AF92BF92DA
:10343000CF92DF92EF920F931F93CF93DF933C01D4
:10344000C091130184E1C89FC02D1124D4E1DC0F89
:10345000D13608F0D0E660911505669580910D058E
:1034600090910E050E94C110182FCD1708F044C08E
:103470008C2E912CF401E05FFD4F9081809114011E
:103480008923C1F1F401EE0FFF1FE05BFE4FC08006
:10349000D12C80E7C81AD108F401EE0FFF1FE05DC0
:1034A000FE4FA1A0B12CE0E2AE1AB108CC9C900175
:1034B000CD9C300D300D1124AA9CC001AB9C900D09
:1034C000900D1124820F931F0E946710082F6091A6
:1034D00012057091130580911405E12E9501A60146
:1034E000F30109950E94CB10462F282F672FC401A6
:1034F0000E942409CF5FB9CF81E0D03608F080E088
:10350000DF91CF911F910F91EF90DF90CF90BF90FF
:10351000AF909F908F907F906F900895CF92DF92A1
:10352000EF92FF920F931F93CF93DF936C01C091A3
:10353000130184E1C89FC02D1124D4E1DC0FD136E2
:1035400008F0D0E660911505669580910D05909183
:103550000E050E94C110182FCD1778F5EC2EF12C16
:10356000F701E05FFD4F908180911401892319F1EB
:10357000F701EE0FFF1FE05DFE4F21A130E020526A
:103580003109F701EE0FFF1FE05BFE4F408150E075
:1035900040575109609112057091130580911405EF
:1035A000012FF60109950E94CB10462F282F672F77
:1035B000C7010E942409CF5FCFCF81E0D03608F049
:1035C00080E0DF91CF911F910F91FF90EF90DF90FE
:1035D000CF900895E9EFF4E08083618324E630E042
:1035E00042E050E0BF0188EE0C941B1FEF92FF9267
:1035F0000F931F93CF93DF937C018B010E94721571
:10360000811119C0E70101151105A1F08091E800B1
:1036100085FD0AC08091E8008E778093E8000E94C3
:103620007215882381F307C089918093F1000150BE
:103630001109E9CF80E0DF91CF911F910F91FF90A9
:10364000EF9008951F93CF93DF93CDB7DEB7AA977E
:103650000FB6F894DEBF0FBECDBFE1EFF4E089EF07
:1036600094E02091F10021938E179F07D1F780916C
:10367000F204833009F461C030F4813071F082309B
:1036800009F49BC0B2C08A3009F487C08B3009F4BA
:103690006CC0893009F0A9C020C08091F104813A42
:1036A00009F0A3C08091E800877F8093E8008091B3
:1036B000F5049091F604892B21F460E28DEC94E0FE
:1036C00003C060E080E090E070E00E942E178091DF
:1036D000E8008B778093E80088C08091F104813204
:1036E00009F083C08091F5049091F604029708F0E8
:1036F0007CC08091E800877F8093E8008091E8009B
:1037000082FD05C08091EF048111F8CF6EC0209139
:10371000F3008091F20090E0922B029731F48091B7
:10372000F100813011F0863021F48091F100809316
:10373000CC048091E8008B7754C08091F104813AE9
:1037400009F053C08091F5049091F604892B09F09B
:103750004CC08091E800877F8093E8008091E8006A
:1037600080FFFCCF8091120137C08091F10481323B
:10377000E1F58091F5049091F604892BB1F58091E3
:10378000E800877F8093E8000E94A5158091F304EC
:10379000809312010E94920328C08091F10481322B
:1037A00021F58091E800877F8093E8000E94A515AD
:1037B0008091F4048093CB0418C08091F104813A85
:1037C000A1F48091E800877F8093E8008091E80071
:1037D00080FFFCCF8091CB048093F1008091E800C2
:1037E0008E778093E8000E94A5158091E80083FF02
:1037F000CEC18091F1049091F204492F50E04A30FB
:10380000510508F0C4C1FA01EA5AFF4F0C94842014
:10381000803821F0823809F0BAC108C08091ED04E7
:103820009091EE04992389F082600FC08091F50495
:103830008F70873008F0ABC18093E9008091EB0076
:1038400085FB882780F91092E9009091E800977F26
:103850009093E8008093F1001092F10065C1282F49
:103860002D7F09F094C1882319F0823061F08FC157
:103870008091F304813009F08AC1933009F080E02F
:103880008093EE042EC08091F30481112AC08091B0
:10389000F5048F702FEF280F263008F078C1809341
:1038A000E9002091EB0020FF1CC0933021F48091AF
:1038B000EB00806214C09091EB0090619093EB005C
:1038C00021E030E0A90102C0440F551F8A95E2F7BC
:1038D0004093EA001092EA008091EB0088608093A8
:1038E000EB001092E9008091E800877F20C18111F0
:1038F0004EC11091F3041F778091E3008078812BF3
:103900008093E3008091E800877F8093E8000E9425
:10391000A5158091E80080FFFCCF8091E3008068CE
:103920008093E300111102C082E001C083E0809324
:10393000EF042DC18058823008F029C18091F30432
:103940009091F4048C3D53E0950779F583E08A83E8
:103950008AE289834FB7F894DE01139620E03EE0B7
:1039600051E2E32FF0E050935700E49120FF03C0B1
:10397000E295EF703F5FEF708E2F90E0EA3010F02D
:10398000C79601C0C0968D939D932F5F243149F750
:103990004FBF8091E800877F8093E8006AE270E083
:1039A000CE0101960E942E17AEC04091F5045091B1
:1039B000F604292F332723303105A9F068F421308C
:1039C000310509F4F3C02230310509F0E0C08BE382
:1039D00090E0EBEFF3E044C02132310521F12232D7
:1039E000310571F1D4C0992781309105A1F058F0CB
:1039F000029709F0CCC0E8E4F4E0E4918E2F90E067
:103A0000E8E4F4E02AC0E4E7F4E0E4918E2F90E0EB
:103A1000E4E7F4E022C0E0E6F4E0E4918E2F90E0E9
:103A2000E0E6F4E01AC04115510509F4C4C0413084
:103A3000510509F0ACC089E090E0E6E2F4E010C086
:103A40004115510509F4BCC04130510509F09FC032
:103A50008BE390E0E0E8F3E003C0009709F497C03F
:103A60002091E800277F2093E8002091F70430910F
:103A7000F8048217930708F49C0140E021153105F2
:103A800089F18091EF04882309F43DC08530D9F194
:103A90008091E80083FD37C08091E80082FD2FC04F
:103AA0008091E80080FFEACF4091F3008091F2001E
:103AB00090E0942B2115310559F08830910540F4A0
:103AC00044914093F1003196215031090196F2CF93
:103AD00041E0089709F040E08091E8008E778093FC
:103AE000E800CCCF4111CDCF0AC08091EF048823EC
:103AF00051F0853041F08091E80083FD04C0809151
:103B0000E80082FFF2CF8091E8008B778093E80095
:103B10003EC08038E1F58091E800877F8093E8001F
:103B20008091F0048093F1008091E8008E7780937B
:103B3000E8000E94A5152BC0811129C08091F304D3
:103B40009091F4049927029714F58091E800877FFB
:103B50008093E8001091F3041093F0040E94A515DF
:103B6000111106C08091E30087FD02C081E001C011
:103B700084E08093EF0442E061EC81E00E94C41590
:103B800042E261EC82E00E94C4158091EF048091D2
:103B9000E80083FF1AC08091E800877F8093E800E7
:103BA0008091EB0080628093EB000FC082E190E097
:103BB000E6E3F4E055CF89E090E0EDE0F4E050CFAB
:103BC00080E490E0EBEBF3E04BCFAA960FB6F894CD
:103BD000DEBF0FBECDBFDF91CF911F9108958093BF
:103BE0001701809111058370809316010E94D013F4
:103BF00083E08093180108958FB7F8944091C4042E
:103C00005091C5046091C6047091C7048FBF409362
:103C10001705509318056093190570931A05809144
:103C20001C05811108C080911105982F937019F01F
:103C30008695869501C080E0909118019130A1F0A1
:103C400028F0923099F0933099F008951092130172
:103C500040930D0550930E0560930F05709310056A
:103C600081E08093180108950C9426090C94EF1DAF
:103C700080911B05882351F046E050E06CE170E034
:103C800081E195E00E94D91F10921B0540910D051E
:103C900050910E0560910F05709110052FB7F894A3
:103CA0008091C4049091C504A091C604B091C7044A
:103CB0002FBF841B950BA60BB70B4097A105B10531
:103CC00010F01092180108951092B90082E08093CC
:103CD000B80008959F92AF92BF92CF92DF92EF9279
:103CE000FF920F931F93CF93DF93B82EEB010E94A7
:103CF000C1176C01C431D10558F0CF3F8FEFD80701
:103D000059F0CE0164E170E00E94421F7B0107C0C0
:103D1000EE24E394F12C03C025E0E22EF12C84E89C
:103D2000A82E94EA992E1092BC009092BC000E949A
:103D3000C1178C018091BC0087FD08C00E94C1178B
:103D4000801B910B8E159F05A8F32AC08091B900A6
:103D5000887F883041F08091B900887F803119F0E8
:103D60000FEF1FEF1FC0B092BB00A092BC000E94DB
:103D7000C1178C018091BC0087FD08C00E94C1174B
:103D8000801B910B8E159F05A8F30AC08091B90086
:103D9000887F883111F0803419F700E010E00EC000
:103DA0000EEF1FEFCF3F8FEFD80709F4BCCFC6014E
:103DB0000E94B2178C179D0708F4B5CFC801DF9198
:103DC000CF911F910F91FF90EF90DF90CF90BF9018
:103DD000AF909F9008950F931F93CF93DF93EB01C4
:103DE0008093BB0084E88093BC000E94C1178C01C3
:103DF0008091BC0087FD0EC0CF3F8FEFD807C1F385
:103E00000E94C117801B910B8C179D0788F38EEFC2
:103E10009FEF0CC02091B900287F81E090E028320C
:103E200011F480E090E0919581959109DF91CF9117
:103E30001F910F910895CF92DF92EF92FF920F930F
:103E40001F93CF93DF936B018A017901B9010E941F
:103E50006A1EE6010C0D1D1DC017D10761F424E98F
:103E60002093BC00DF91CF911F910F91FF90EF90B5
:103E7000DF90CF90089597FDF2CFB70189910E940E
:103E8000EB1EEACFAA1BBB1B51E107C0AA1FBB1F39
:103E9000A617B70710F0A61BB70B881F991F5A95D6
:103EA000A9F780959095BC01CD0108958F929F92BE
:103EB000AF92BF92CF92DF92EF92FF92CF93DF93B8
:103EC000EC01688179818A819B8161157105810589
:103ED000910521F464E279ED8BE597E02DE133EF74
:103EE00041E050E00E940D2049015A019B01AC01C4
:103EF000A7EAB1E40E942C206B017C01ACEEB4EF88
:103F0000A50194010E943A20DC01CB018C0D9D1D7E
:103F1000AE1DBF1DB7FF03C00197A109B04888833C
:103F20009983AA83BB839F77DF91CF91FF90EF9016
:103F3000DF90CF90BF90AF909F908F9008950E9498
:103F4000561F089580E091E00E94561F0895A0E05A
:103F5000B0E08093000190930101A0930201B0931F
:103F600003010895FB01DC0102C005900D92415050
:103F70005040D8F70895DC01CB01FC01F999FECF40
:103F800006C0F2BDE1BDF89A319600B40D924150E1
:103F90005040B8F70895F999FECF92BD81BDF89AC7
:103FA000992780B50895A8E1B0E042E050E00C9474
:103FB000BD1FDC01A40FB51F4150504048F0CB019C
:103FC000840F951F2E910E94EA1F41505040D0F758
:103FD0000895262FF999FECF92BD81BDF89A0197D9
:103FE00000B4021639F01FBA20BD0FB6F894FA9A41
:103FF000F99A0FBE08950396272F0E94EA1F0E9488
:10400000E91F252F0E94EA1F242F0C94EA1F019616
:10401000272F0E94EA1F0C94E91F052E97FB1EF420
:1040200000940E94242057FD07D00E943F2007FCE7
:1040300003D04EF40C942420509540953095219552
:104040003F4F4F4F5F4F08959095809570956195C4
:104050007F4F8F4F9F4F08950E946120A59F900D25
:10406000B49F900DA49F800D911D11240895B7FF5A
:104070000C942C200E942C20821B930B0895A1E20B
:104080001A2EAA1BBB1BFD010DC0AA1FBB1FEE1FD2
:10409000FF1FA217B307E407F50720F0A21BB30B1D
:1040A000E40BF50B661F771F881F991F1A9469F799
:1040B00060957095809590959B01AC01BD01CF01F5
:1040C0000895A29FB001B39FC001A39F700D811DF1
:1040D0001124911DB29F700D811D1124911D089511
:1040E00097FB072E16F4009407D077FD09D00E94A5
:1040F000421F07FC05D03EF4909581959F4F08958F
:10410000709561957F4F0895EE0FFF1F0590F49114
:10411000E02D0994FB01DC0104C08D910190801910
:1041200021F441505040C8F7881B990B0895F8942A
:02413000FFCFBF
:10413200010000002B132E132A132813291327130F
:1041420039050100FF00FFFF0300FFFF67663635F8
:1041520034979694F7F6F5F4003131295A1B750A13
:10416200000102030405060708090A0B0C0D0E0FD5
:10417200101112131415161718191A1B1C1D1E1FC5
:1041820000002000400060008000A000C000E000AD
:1041920000152015401560158015A015C015E015F5
:1041A200002A202A402A602A802AA02AC02AE02A3D
:1041B20000402040404060408040A040C040E0407D
:1041C20000000000000000000000000000000000ED
:1041D20000000000000000000000000000000000DD
:1041E20000000000000000000000000000000000CD
:1041F20000000000000000000000000000000000BD
:1042020000000000000000000000000000000000AC
:10421200000000000000000000000000000000009C
:10422200000000000000000000000000000000008C
:10423200000000000000000000000000000000007C
:10424200040404040404040404040404040404042C
:10425200040404040404040404040404040404041C
:10426200000000000000000000000000000000004C
:10427200000000000000000000000000000000003C
:10428200000000000000000000000000000000002C
:10429200000000000000000000000000000000001C
:00000001FF
